 mouhid

 Timestamp is 4fb05c72 (Mon May 14 13:14:26 2012)

 Preferred load address is 10000000

 Start         Length     Name                   Class
 0001:00000000 00000004H .CRT$XCA                CODE
 0001:00000004 00000004H .CRT$XCZ                CODE
 0001:00000008 00000004H .CRT$XIA                CODE
 0001:0000000c 00000004H .CRT$XIZ                CODE
 0001:00000010 00000004H .CRT$XPA                CODE
 0001:00000014 00000004H .CRT$XPZ                CODE
 0001:00000018 00000004H .CRT$XTA                CODE
 0001:0000001c 00000004H .CRT$XTZ                CODE
 0001:00000020 0000056eH .rdata                  CODE
 0001:00000590 00000023H .rdata$debug            CODE
 0001:000005b4 000023d0H .text                   CODE
 0001:00002984 00000018H .xdata                  CODE
 0001:0000299c 00000028H .idata$2                CODE
 0001:000029c4 00000014H .idata$3                CODE
 0001:000029d8 00000094H .idata$4                CODE
 0001:00002a6c 000000aaH .idata$6                CODE
 0001:00002b20 0000006eH .edata                  CODE
 0002:00000000 00000094H .idata$5                DATA
 0002:00000098 00000454H .data                   DATA
 0002:000004ec 0000001cH .bss                    DATA
 0003:00000000 00000118H .pdata                  DATA

  Address         Publics by Value              Rva+Base       Lib:Object

 0000:00000000       ___safe_se_handler_count   00000000     <absolute>
 0000:00000000       ___safe_se_handler_table   00000000     <absolute>
 0001:00000000       __xc_a                     10001000     corelib0:crt0init.obj
 0001:00000004       __xc_z                     10001004     corelib0:crt0init.obj
 0001:00000008       __xi_a                     10001008     corelib0:crt0init.obj
 0001:0000000c       __xi_z                     1000100c     corelib0:crt0init.obj
 0001:00000010       __xp_a                     10001010     corelib0:crt0init.obj
 0001:00000014       __xp_z                     10001014     corelib0:crt0init.obj
 0001:00000018       __xt_a                     10001018     corelib0:crt0init.obj
 0001:0000001c       __xt_z                     1000101c     corelib0:crt0init.obj
 0001:0000005c       ??_C@_1BK@BJEDGIOP@?$AA?$CF?$AAs?$AA?3?$AA?5?$AAD?$AAe?$AAt?$AAa?$AAc?$AAh?$AA?$AN?$AA?6?$AA?$AA@ 1000105c     mouhid.obj
 0001:00000078       ??_C@_1CG@JHDABJCF@?$AAM?$AAo?$AAu?$AAs?$AAe?$AAD?$AAe?$AAt?$AAa?$AAc?$AAh?$AAe?$AAd?$AAE?$AAv?$AAe?$AAn?$AAt?$AA?$AA@ 10001078     mouhid.obj
 0001:000000a0       ??_C@_1CG@NNBNONKD@?$AAM?$AAo?$AAu?$AAs?$AAe?$AAA?$AAt?$AAt?$AAa?$AAc?$AAh?$AAe?$AAd?$AAE?$AAv?$AAe?$AAn?$AAt?$AA?$AA@ 100010a0     mouhid.obj
 0001:000000c8       ??_C@_1BK@LFPGKGAH@?$AA?$CF?$AAs?$AA?3?$AA?5?$AAA?$AAt?$AAt?$AAa?$AAc?$AAh?$AA?$AN?$AA?6?$AA?$AA@ 100010c8     mouhid.obj
 0001:000000e4       ??_C@_1CA@OKFACCGM@?$AAM?$AAO?$AAU?$AAH?$AAI?$AAD?$AA?5?$AAD?$AAl?$AAl?$AAE?$AAn?$AAt?$AAr?$AAy?$AA?$AA@ 100010e4     mouhid.obj
 0001:00000108       ??_C@_1EG@HEENEOMI@?$AA?$CF?$AAs?$AA?3?$AA?5?$AAF?$AAa?$AAi?$AAl?$AAe?$AAd?$AA?5?$AAc?$AAr?$AAe?$AAa?$AAt?$AAi?$AAn?$AAg?$AA?5?$AAm?$AAo?$AAu?$AAs?$AAe?$AA?5?$AAt?$AAh?$AAr?$AAe?$AAa?$AAd@ 10001108     mouhid.obj
 0001:00000150       ??_C@_1DE@IIKINMKE@?$AA?$CF?$AAs?$AA?3?$AA?5?$AAL?$AAo?$AAc?$AAa?$AAl?$AAA?$AAl?$AAl?$AAo?$AAc?$AA?5?$AAe?$AAr?$AAr?$AAo?$AAr?$AA?3?$AA?$CF?$AAd?$AA?$AN?$AA?6?$AA?$AA@ 10001150     mouhid.obj
 0001:00000188       ??_C@_1FK@FNONLNGN@?$AA?$CF?$AAs?$AA?3?$AA?5?$AAD?$AAE?$AAB?$AAU?$AAG?$AAC?$AAH?$AAK?$AA?5?$AAf?$AAa?$AAi?$AAl?$AAe?$AAd?$AA?5?$AAi?$AAn?$AA?5?$AAf?$AAi?$AAl?$AAe?$AA?5?$AA?$CF?$AAs?$AA?5?$AAa@ 10001188     mouhid.obj
 0001:000001e8       ??_C@_1JI@NHLALKPD@?$AAC?$AA?3?$AA?2?$AAW?$AAI?$AAN?$AAC?$AAE?$AAR?$AAO?$AAO?$AAT?$AAS?$AA?2?$AAT?$AAo?$AAp?$AAa?$AAz?$AA?2?$AAW?$AAI?$AAN?$AAC?$AAE?$AA6?$AA0?$AA0?$AA?2?$AAP?$AAL?$AAA@ 100011e8     mouhid.obj
 0001:00000280       ??_C@_1CA@LBENOBMA@?$AAH?$AAI?$AAD?$AAD?$AAe?$AAv?$AAi?$AAc?$AAe?$AAA?$AAt?$AAt?$AAa?$AAc?$AAh?$AA?$AA@ 10001280     mouhid.obj
 0001:000002a0       ??_C@_1CK@EJMAOEFN@?$AA?$CF?$AAs?$AA?3?$AA?5?$AAE?$AAx?$AAi?$AAt?$AAi?$AAn?$AAg?$AA?5?$AAt?$AAh?$AAr?$AAe?$AAa?$AAd?$AA?$AN?$AA?6?$AA?$AA@ 100012a0     mouhid.obj
 0001:000002d0       ??_C@_1GM@KAMEMAIN@?$AA?$CF?$AAs?$AA?3?$AA?5?$AAG?$AAe?$AAt?$AAI?$AAn?$AAt?$AAe?$AAr?$AAr?$AAu?$AAp?$AAt?$AAR?$AAe?$AAp?$AAo?$AAr?$AAt?$AA?5?$AAr?$AAe?$AAt?$AAu?$AAr?$AAn?$AAe?$AAd?$AA?5@ 100012d0     mouhid.obj
 0001:0000033c       ??_C@_1CA@FPPCBODG@?$AAM?$AAo?$AAu?$AAs?$AAe?$AAT?$AAh?$AAr?$AAe?$AAa?$AAd?$AAP?$AAr?$AAo?$AAc?$AA?$AA@ 1000133c     mouhid.obj
 0001:0000035c       ??_C@_1DG@LDJIBABC@?$AA?$CF?$AAs?$AA?3?$AA?5?$AAU?$AAn?$AAh?$AAa?$AAn?$AAd?$AAl?$AAe?$AAd?$AA?5?$AAm?$AAe?$AAs?$AAs?$AAa?$AAg?$AAe?$AA?5?$AA?$CF?$AAu?$AA?$AN?$AA?6?$AA?$AA@ 1000135c     mouhid.obj
 0001:00000398       ??_C@_1FC@MGAKAGG@?$AA?$CF?$AAs?$AA?3?$AA?5?$AAR?$AAe?$AAc?$AAe?$AAi?$AAv?$AAe?$AAd?$AA?5?$AAi?$AAn?$AAv?$AAa?$AAl?$AAi?$AAd?$AA?5?$AAs?$AAt?$AAr?$AAu?$AAc?$AAt?$AAu?$AAr?$AAe?$AA?5?$AAp@ 10001398     mouhid.obj
 0001:000003ec       ??_C@_1CO@LBEHPIKP@?$AAH?$AAI?$AAD?$AAD?$AAe?$AAv?$AAi?$AAc?$AAe?$AAN?$AAo?$AAt?$AAi?$AAf?$AAi?$AAc?$AAa?$AAt?$AAi?$AAo?$AAn?$AAs?$AA?$AA@ 100013ec     mouhid.obj
 0001:0000041c       ??_C@_1BA@LEPJIIOK@?$AAU?$AAn?$AAk?$AAn?$AAo?$AAw?$AAn?$AA?$AA@ 1000141c     mouhid.obj
 0001:0000042c       ??_C@_1CG@NEOOBILK@?$AAA?$AAl?$AAl?$AAo?$AAc?$AAa?$AAt?$AAe?$AAU?$AAs?$AAa?$AAg?$AAe?$AAL?$AAi?$AAs?$AAt?$AAs?$AA?$AA@ 1000142c     mouhid.obj
 0001:00000458       ??_C@_1CG@EAKONFHH@?$AAP?$AAr?$AAo?$AAc?$AAe?$AAs?$AAs?$AAM?$AAo?$AAu?$AAs?$AAe?$AAR?$AAe?$AAp?$AAo?$AAr?$AAt?$AA?$AA@ 10001458     mouhid.obj
 0001:00000480       ??_C@_1GK@KPHAPAKG@?$AA?$CF?$AAs?$AA?3?$AA?5?$AAB?$AAa?$AAd?$AA?5?$AAp?$AAh?$AAy?$AAs?$AAi?$AAc?$AAa?$AAl?$AA?5?$AAm?$AAa?$AAx?$AA?1?$AAm?$AAi?$AAn?$AA?5?$AAf?$AAo?$AAr?$AA?5?$AAm?$AAo?$AAu@ 10001480     mouhid.obj
 0001:000004ec       ??_C@_1CA@LFKNIOKP@?$AAG?$AAe?$AAt?$AAA?$AAx?$AAi?$AAs?$AAM?$AAo?$AAv?$AAe?$AAm?$AAe?$AAn?$AAt?$AA?$AA@ 100014ec     mouhid.obj
 0001:00000510       ??_C@_1GI@FFADIIEP@?$AA?$CF?$AAs?$AA?3?$AA?5?$AAH?$AAI?$AAD?$AA?3?$AA?5?$AAd?$AAx?$AA?5?$AA?$CF?$AA4?$AAd?$AA?0?$AA?5?$AAd?$AAy?$AA?5?$AA?$CF?$AA4?$AAd?$AA?0?$AA?5?$AAd?$AAw?$AAD?$AAa?$AAt?$AAa?$AA?5@ 10001510     mouhid.obj
 0001:00000578       ??_C@_1BG@PCLEONCF@?$AAM?$AAo?$AAu?$AAs?$AAe?$AAE?$AAv?$AAe?$AAn?$AAt?$AA?$AA@ 10001578     mouhid.obj
 0001:000005b4       DllEntry                   100015b4 f   mouhid.obj
 0001:00000738       HIDDeviceAttach            10001738 f   mouhid.obj
 0001:00000ce8       HIDDeviceNotifications     10001ce8 f   mouhid.obj
 0001:00001908       ?FreeHidMouse@@YAXPAU_HID_MOUSE@@@Z 10002908 f   mouhid.obj
 0001:00001e58       SetEvent                   10002e58 f i mouhid.obj
 0001:00001e90       GetCurrentThread           10002e90 f i mouhid.obj
 0001:00001ea8       HidP_MaxUsageListLength    10002ea8 f   hidparse:HIDPARSE.dll
 0001:00001eb8       HidP_GetCaps               10002eb8 f   hidparse:HIDPARSE.dll
 0001:00001ec8       HidP_GetSpecificValueCaps  10002ec8 f   hidparse:HIDPARSE.dll
 0001:00001ed8       HidP_UsageListDifference   10002ed8 f   hidparse:HIDPARSE.dll
 0001:00001ee8       HidP_GetUsages             10002ee8 f   hidparse:HIDPARSE.dll
 0001:00001ef8       HidP_GetScaledUsageValue   10002ef8 f   hidparse:HIDPARSE.dll
 0001:00001f08       DriverMouseHookInitialize  10002f08 f   MouHidStd:StandardMouse.obj
 0001:00001f30       DriverMouseHook            10002f30 f   MouHidStd:StandardMouse.obj
 0001:00001f58       CloseHandle                10002f58 f   coredll:COREDLL.dll
 0001:00001f68       CreateEventW               10002f68 f   coredll:COREDLL.dll
 0001:00001f78       DisableThreadLibraryCalls  10002f78 f   coredll:COREDLL.dll
 0001:00001f88       NKDbgPrintfW               10002f88 f   coredll:COREDLL.dll
 0001:00001f98       RegisterDbgZones           10002f98 f   coredll:COREDLL.dll
 0001:00001fa8       CreateThread               10002fa8 f   coredll:COREDLL.dll
 0001:00001fb8       GetLastError               10002fb8 f   coredll:COREDLL.dll
 0001:00001fc8       LocalAlloc                 10002fc8 f   coredll:COREDLL.dll
 0001:00001fd8       EventModify                10002fd8 f   coredll:COREDLL.dll
 0001:00001fe8       LocalFree                  10002fe8 f   coredll:COREDLL.dll
 0001:00001ff8       SetThreadPriority          10002ff8 f   coredll:COREDLL.dll
 0001:00002008       WaitForSingleObject        10003008 f   coredll:COREDLL.dll
 0001:00002018       mouse_event                10003018 f   coredll:COREDLL.dll
 0001:00002028       LocalSize                  10003028 f   coredll:COREDLL.dll
 0001:00002038       _DllEntryCRTStartup        10003038 f   corelib0:pegdentry.obj
 0001:000020a8       __security_init_cookie     100030a8 f   corelib0:seccinit.obj
 0001:00002170       __GSHandlerCheck           10003170 f   corelib0:gshandler.obj
 0001:000021b8       __GSHandlerCheckCommon     100031b8 f   corelib0:gshandler.obj
 0001:00002260       __security_check_cookie    10003260 f   corelib0:armsecgs.obj
 0001:00002274       __gsfailure                10003274 f   corelib0:armsecgs.obj
 0001:000022b8       exit                       100032b8 f   corelib0:cexit.obj
 0001:00002438       _exit                      10003438 f   corelib0:cexit.obj
 0001:0000245c       _cexit                     1000345c f   corelib0:cexit.obj
 0001:00002478       _c_exit                    10003478 f   corelib0:cexit.obj
 0001:00002494       GetCurrentProcess          10003494 f i corelib0:cexit.obj
 0001:000024ac       _initterm                  100034ac f   corelib0:crt0dat.obj
 0001:00002500       _cinit                     10003500 f   corelib0:crt0dat.obj
 0001:0000253c       _onexit                    1000353c f   corelib0:onexit.obj
 0001:00002840       atexit                     10003840 f   corelib0:onexit.obj
 0001:00002894       memcpy                     10003894 f   corelib1:COREDLL.dll
 0001:000028a4       __security_gen_cookie2     100038a4 f   corelib1:COREDLL.dll
 0001:000028b4       __report_gsfailure         100038b4 f   corelib1:COREDLL.dll
 0001:000028c4       free                       100038c4 f   corelib1:COREDLL.dll
 0001:000028d4       __C_specific_handler       100038d4 f   corelib1:COREDLL.dll
 0001:000028e4       malloc                     100038e4 f   corelib1:COREDLL.dll
 0001:000028f4       realloc                    100038f4 f   corelib1:COREDLL.dll
 0001:00002904       _msize                     10003904 f   corelib1:COREDLL.dll
 0001:00002914       DeleteCriticalSection      10003914 f   coredll:COREDLL.dll
 0001:00002924       InterlockedExchange        10003924 f   coredll:COREDLL.dll
 0001:00002934       TerminateProcess           10003934 f   coredll:COREDLL.dll
 0001:00002944       EnterCriticalSection       10003944 f   coredll:COREDLL.dll
 0001:00002954       InterlockedCompareExchange 10003954 f   coredll:COREDLL.dll
 0001:00002964       InitializeCriticalSection  10003964 f   coredll:COREDLL.dll
 0001:00002974       LeaveCriticalSection       10003974 f   coredll:COREDLL.dll
 0001:0000299c       __IMPORT_DESCRIPTOR_HIDPARSE 1000399c     hidparse:HIDPARSE.dll
 0001:000029b0       __IMPORT_DESCRIPTOR_COREDLL 100039b0     coredll:COREDLL.dll
 0001:000029c4       __NULL_IMPORT_DESCRIPTOR   100039c4     hidparse:HIDPARSE.dll
 0002:00000000       __imp_WaitForSingleObject  10004000     coredll:COREDLL.dll
 0002:00000004       __imp_InitializeCriticalSection 10004004     coredll:COREDLL.dll
 0002:00000008       __imp_InterlockedCompareExchange 10004008     coredll:COREDLL.dll
 0002:0000000c       __imp_EnterCriticalSection 1000400c     coredll:COREDLL.dll
 0002:00000010       __imp_TerminateProcess     10004010     coredll:COREDLL.dll
 0002:00000014       __imp_InterlockedExchange  10004014     coredll:COREDLL.dll
 0002:00000018       __imp_DeleteCriticalSection 10004018     coredll:COREDLL.dll
 0002:0000001c       __imp_CloseHandle          1000401c     coredll:COREDLL.dll
 0002:00000020       __imp_CreateEventW         10004020     coredll:COREDLL.dll
 0002:00000024       __imp_DisableThreadLibraryCalls 10004024     coredll:COREDLL.dll
 0002:00000028       __imp_NKDbgPrintfW         10004028     coredll:COREDLL.dll
 0002:0000002c       __imp_RegisterDbgZones     1000402c     coredll:COREDLL.dll
 0002:00000030       __imp_CreateThread         10004030     coredll:COREDLL.dll
 0002:00000034       __imp_GetLastError         10004034     coredll:COREDLL.dll
 0002:00000038       __imp_LocalAlloc           10004038     coredll:COREDLL.dll
 0002:0000003c       __imp_EventModify          1000403c     coredll:COREDLL.dll
 0002:00000040       __imp_LocalFree            10004040     coredll:COREDLL.dll
 0002:00000044       __imp_SetThreadPriority    10004044     coredll:COREDLL.dll
 0002:00000048       __imp_LeaveCriticalSection 10004048     coredll:COREDLL.dll
 0002:0000004c       __imp_mouse_event          1000404c     coredll:COREDLL.dll
 0002:00000050       __imp_LocalSize            10004050     coredll:COREDLL.dll
 0002:00000054       __imp_memcpy               10004054     corelib1:COREDLL.dll
 0002:00000058       __imp___security_gen_cookie2 10004058     corelib1:COREDLL.dll
 0002:0000005c       __imp___report_gsfailure   1000405c     corelib1:COREDLL.dll
 0002:00000060       __imp_free                 10004060     corelib1:COREDLL.dll
 0002:00000064       __imp___C_specific_handler 10004064     corelib1:COREDLL.dll
 0002:00000068       __imp_malloc               10004068     corelib1:COREDLL.dll
 0002:0000006c       __imp_realloc              1000406c     corelib1:COREDLL.dll
 0002:00000070       __imp__msize               10004070     corelib1:COREDLL.dll
 0002:00000074       \177COREDLL_NULL_THUNK_DATA 10004074     coredll:COREDLL.dll
 0002:00000078       __imp_HidP_GetScaledUsageValue 10004078     hidparse:HIDPARSE.dll
 0002:0000007c       __imp_HidP_GetUsages       1000407c     hidparse:HIDPARSE.dll
 0002:00000080       __imp_HidP_UsageListDifference 10004080     hidparse:HIDPARSE.dll
 0002:00000084       __imp_HidP_GetSpecificValueCaps 10004084     hidparse:HIDPARSE.dll
 0002:00000088       __imp_HidP_GetCaps         10004088     hidparse:HIDPARSE.dll
 0002:0000008c       __imp_HidP_MaxUsageListLength 1000408c     hidparse:HIDPARSE.dll
 0002:00000090       \177HIDPARSE_NULL_THUNK_DATA 10004090     hidparse:HIDPARSE.dll
 0002:00000098       dpCurSettings              10004098     mouhid.obj
 0002:000004e4       __security_cookie          100044e4     corelib0:seccinit.obj
 0002:000004e8       __security_cookie_complement 100044e8     corelib0:seccinit.obj
 0002:000004f8       _exitflag                  100044f8     corelib0:cexit.obj
 0002:000004fc       __onexitend                100044fc     <common>
 0002:00000500       __onexitbegin              10004500     <common>
 0002:00000504       g_pcsExit                  10004504     <common>

 entry point at        0001:00002038

 Static symbols

 0001:00000a74       ?MouseThreadProc@@YAKPAX@Z 10001a74 f   mouhid.obj
 0001:00000ea0       ?AllocateUsageLists@@YAHPAU_HID_MOUSE@@I@Z 10001ea0 f   mouhid.obj
 0001:00001088       ?DetermineWheelUsage@@YAXPAU_HID_MOUSE@@@Z 10002088 f   mouhid.obj
 0001:000011cc       ?SetButtonFlags@@YAXPAKPAGKPBKK@Z 100021cc f   mouhid.obj
 0001:00001340       ?ProcessMouseReport@@YAXPAU_HID_MOUSE@@PADK@Z 10002340 f   mouhid.obj
 0001:00001674       ?GetAxisMovement@@YAJPAU_HID_MOUSE@@GPADKPAJ@Z 10002674 f   mouhid.obj
 0001:0000180c       ?MouseEvent@@YAXKKKK@Z     1000280c f   mouhid.obj
 0001:000019dc       ?ValidateHidMouse@@YAXPAU_HID_MOUSE@@@Z 100029dc f   mouhid.obj
 0001:000022dc       doexit                     100032dc f   corelib0:cexit.obj
 0001:00002598       lockexit                   10003598 f   corelib0:onexit.obj
 0001:00002634       unlockexit                 10003634 f   corelib0:onexit.obj
 0001:00002660       _onexit_nolock             10003660 f   corelib0:onexit.obj
